S011000048656E64694374726C2E7372656396
S11300000C9434000C9451000C9451000C94510045
S11300100C9451000C9451000C9451000C94510018
S11300200C9451000C9451000C9451000C94510008
S11300300C9451000C94CC060C9451000C94510077
S11300400C9451000C9451000C9485070C947B077C
S11300500C9471070C9482000C9451000C94510080
S11300600C9451000C94510011241FBECFEFD8E022
S1130070DEBFCDBF12E0A0E0B1E0E8E5FCE102C0E4
S113008005900D92AC34B107D9F722E0ACE4B2E0AC
S113009001C01D92A13DB207E1F70E94D1020C9468
S11300A02A0E0C94000090935D0280935C0228E178
S11300B031E041E050E060E170E08EE492E00E94C3
S11300C01E01E4E6F0E080818E7F8083EAE7F0E0C1
S11300D08081876880830895ECE7F0E09081907FC9
S11300E090648F70982B9083EAE7F0E09081986495
S11300F0908380935E0281E090E090934D02809320
S11301004C0208951F920F920FB60F9211242F9351
S11301103F934F935F936F937F938F939F93AF938B
S1130120BF93EF93FF93CF93DF93CDB7DEB72597BC
S1130130DEBFCDBF10924D0210924C028091780028
S11301402091790090917A00906190937A0092E0E6
S1130150998390915E029A8390E0922B9C838B8387
S1130160BE016F5F7F4F80915C0290915D020E949F
S113017063018EE492E00E94F201892B51F4BE01E6
S11301806B5F7F4F8EE492E00E94AC018D810E94F0
S11301906C000F900F900F900F900F90DF91CF9104
S11301A0FF91EF91BF91AF919F918F917F916F914B
S11301B05F914F913F912F910F900FBE0F901F9021
S11301C01895CF93DF931F92CDB7DEB789838091C3
S11301D04C0290914D02892B21F489810E946C007C
S11301E007C0BE016F5F7F4F8EE492E00E946301FF
S11301F00F90DF91CF910895F89480915F029091D0
S1130200600201969093600280935F02089580914A
S11302105F0290916002892B81F080915F0290913E
S1130220600201979093600280935F0280915F0265
S113023090916002892B09F4789408958F929F928B
S1130240AF92BF92CF92DF92EF92FF920F931F93E0
S1130250CF93DF93EC017B014A015901198618867B
S11302601B861A861F821E827B836A835D834C836E
S1130270CB01880F991F0E94D1089983888300E0DD
S113028010E00E151F0581F0C801880F991FC88062
S1130290D980C80ED91EC4010E94D108F6019183E9
S11302A080830F5F1F4FEDCFBD86AC86DF91CF916A
S11302B01F910F91FF90EF90DF90CF90BF90AF9080
S11302C09F908F9008950F931F93CF93DF93EC012A
S11302D08B010E94FC002E813F818A819B8128171B
S11302E0390768F5D8019D01201B310B8C819D8154
S11302F02817390780F4E885F9854D91EE0FFF1F23
S113030088819981E80FF91F80819181FC01E20FB6
S1130310F31F4083E8CF888599850196998788875C
S11303208E819F8101969F838E83288539858A815A
S11303309B812817390731F41986188603C0C0E059
S1130340D0E002C0C1E0D0E00E940701CE01DF91FD
S1130350CF911F910F9108950F931F93CF93DF9324
S1130360EC018B010E94FC008E819F81892B69F135
S1130370D801CD01801B910B2C813D8182179307FD
S113038080F4EA85FB85EE0FFF1F28813981E20F97
S1130390F31F20813181F901E80FF91F80818D93CA
S11303A0E8CF8A859B8501969B878A878E819F816A
S11303B001979F838E832A853B858A819B81281799
S11303C0390731F41B861A8603C0C0E0D0E002C0AE
S11303D0C1E0D0E00E940701CE01DF91CF911F91CF
S11303E00F910895CF93DF93EC010E94FC000E80DF
S11303F0DF81C02D0E94070181E090E0CD2B11F038
S113040080E090E0DF91CF9108958FEF8093B80062
S11304101092B900089594EA9093BC009091BC00A6
S113042097FFFCCF9091B900987F983019F081E242
S113043091E017C0880F682B6093BB0084E8809319
S1130440BC008091BC0087FFFCCF8091B900887FFD
S1130450883129F4FA01240F351F94E805C081E39B
S113046091E00E946B0B14C0E217F30789F08191AD
S11304708093BB009093BC008091BC0087FFFCCFAD
S11304808091B900887F883279F383E491E0E9CFE1
S113049084E98093BC0008950F931F93CF93DF9357
S11304A000D000D0CDB7DEB78C0190936602809364
S11304B065028091140190911501A0911601B091EB
S11304C0170189839A83AB83BC8380916D029091D9
S11304D06E02892BE9F0E1E0F0E00115110511F459
S11304E0E0E0F0E0EE0FFF1F81E090E08C0F9D1F35
S11304F0E80FF91F81818F9380818F9386E591E0C6
S11305009F938F930E94550B0F900F900F900F9015
S113051061E070E0012B11F460E070E087E090E0AE
S11305200F900F900F900F90DF91CF911F910F912B
S11305300C94AD060F931F93CF93DF9300D0CDB7E8
S1130540DEB78C01809361021093620280916D0288
S113055090916E02892B61F01F930F938FE691E0C7
S11305609F938F930E94550B0F900F900F900F90B5
S113057019821A8242E050E0BE016F5F7F4FC801CA
S11305800E9491069C01AE014F5F5F4F60E080E6E0
S11305900E940B020F900F90DF91CF911F910F914A
S11305A00895CF93DF93CDB7DEB76B970FB6F8946A
S11305B0DEBF0FBECDBFF894A8950FB6F894A895EA
S11305C080916000886180936000109260000FBE8B
S11305D02CE131E044E050E068E070E087EB92E029
S11305E00E941E0140E052EC61E070E087EB92E073
S11305F00E94C90742E06FEF76EF87EB92E00E941A
S1130600410787EB92E00E9453000E9405020E947A
S1130610A50686E091E09093CC028093CB0281E220
S113062092E09F938F9386E292E09F938F9387E863
S113063091E09F938F930E94550B1D8A1E8A1F8AF7
S113064043E050E0BE016B5E7F4F80E090E00E948B
S113065098069C01AE014B5E5F4F60E080E60E940D
S11306600B026091CB027091CC028DE090E00E946D
S1130670190B6091CB027091CC028AE090E00E9449
S1130680190B6091CB027091CC028AE390E00E9436
S1130690190B60E070E080E00E94590760E070E0B0
S11306A082E00E94590781E090E00E944C02789415
S11306B00F900F900F900F900F900F90F12C212C12
S11306C0312C68EE462E63E0562E612C712C73EBB0
S11306D0A72E71E0B72EE0EB8E2EE1E09E2E87EB85
S11306E092E00E94F201892B09F016C3BE016F5EED
S11306F07F4F87EB92E00E94AC018989823009F434
S113070021C2833009F44CC2813009F005C38A89BF
S113071020916F0230917002AE014F5F5F4FFA017A
S1130720E20FF31F10828D3009F0F7C1598F488F03
S11307301092700210926F02EF2C8F2D90E0880FB0
S1130740991F9C01255E3D4F3B8F2A8F56E9C52E8C
S113075051E0D52E088D198DF80180818823D9F0B8
S113076090E00E94110B9C01C8010196998F888F1B
S11307702035310509F055C0F80121812F3329F4C2
S11307800E5F1F4F198F088F31C030E0205331099D
S11307902A303105F0F060E177E281E00E945907E8
S11307A06091CB027091CC028DE090E00E94190B15
S11307B06091CB027091CC028AE090E00E94190B08
S11307C06091CB027091CC028AE390E00E94190BF5
S11307D063C24AE050E0BE01685E7F4F0E94F209A6
S11307E0E1E0FE12BAC0CB010E949A026091CB02F2
S11307F07091CC028DE090E00E94190B6091CB02C5
S11308007091CC028AE090E00E94190B8091620200
S11308108F93809161028F932EE831E03F932F9361
S11308205CC123353105B1F5F80121812F3329F459
S11308300E5F1F4F198F088F14C030E02053310909
S11308402A30310508F0A7CF4AE050E0BE01685EC7
S11308507F4F0E94F209E1E0FE127FC0CB010E94AB
S11308604C026091CB027091CC028DE090E00E942A
S1130870190B6091CB027091CC028AE090E00E9447
S1130880190B809166028F93809165028F9324EAFD
S113089031E0C4CF2235310509F072C0F80121815D
S11308A02F3309F475C030E0205331092A30310563
S11308B008F071CF4AE050E0BE01685E7F4F0E94AD
S11308C0F2096130710519F5F11047C08FEF9FE00F
S11308D00E949A0280E090E00E944C026091CB0258
S11308E07091CC028DE090E00E94190B6091CB02D4
S11308F07091CC028AE090E00E94190B9F928F9233
S11309000E94550B0F900F90EE24E39423CF672B96
S113091009F020CF91E0F91220C08FEF9FE00E94F0
S11309209A0280E090E00E944C026091CB027091A8
S1130930CC028DE090E00E94190B6091CB02709183
S1130940CC028AE090E00E94190B9F928F920E9441
S1130950550B0F900F90E12CFDCE6091CB0270915E
S1130960CC028DE090E00E94190B6091CB02709153
S1130970CC028AE090E00E94190BDF92CF92C8C0AB
S11309802434310509F045C0F80121812F33E1F405
S11309900E5F1F4F198F088F6091CB027091CC02AC
S11309A08DE090E00E94190B6091CB027091CC0213
S11309B08AE090E00E94190B81E0E81280E01F9227
S11309C08F932AEA31E02ACF30E0205331092A30CC
S11309D0310508F0E0CE4AE050E0BE01685E7F4F8A
S11309E00E94F20970936E0260936D026091CB02D3
S11309F07091CC028DE090E00E94190B6091CB02C3
S1130A007091CC028AE090E00E94190B9F928F9221
S1130A107FC029343105E1F4F80181818F3309F075
S1130A2099CE0E5F1F4F198F088F6091CB02709182
S1130A30CC028DE090E00E94190B6091CB02709182
S1130A40CC028AE090E00E94190B26E232E01EC03C
S1130A5026353105F1F4F80181818F3309F07ACE1E
S1130A600E5F1F4F198F088F6091CB027091CC02DB
S1130A708DE090E00E94190B6091CB027091CC0242
S1130A808AE090E00E94190B21E232E03F932F9319
S1130A9022C02435310541F5F80181818F3309F0F5
S1130AA059CE0E5F1F4F198F088FEA8DFB8D108171
S1130AB001816091CB027091CC028DE090E00E94A4
S1130AC0190B6091CB027091CC028AE090E00E94F5
S1130AD0190B0F931F93BF92AF920E94550B0F9067
S1130AE00F900F900F9036CE6091CB027091CC0294
S1130AF08DE090E00E94190B6091CB027091CC02C2
S1130B008AE090E00E94190B29EB31E03F932F9388
S1130B100E94550B0F900F901DCE8A3009F4FCC033
S1130B202F30310538F42F5F3F4F309370022093FC
S1130B306F0280836091CB027091CC0290E00E949E
S1130B40190BEAC08A890B891C89811116C080910E
S1130B506302909164020817190709F4DDC0F110CB
S1130B6007C0C801880F991F880F991F0E949A0215
S1130B701093640200936302CFC0823009F0CCC0AA
S1130B8010936C0200936B0281E090E001301240FC
S1130B9014F480E090E090936A0280936902BCC0F0
S1130BA08A89813049F118F08230A9F1B5C021E079
S1130BB0F21203C024EF31E002C028EE33E08101D9
S1130BC081E00827232819F462E370E00BC0225364
S1130BD03109A8EEB3E00E94B708A30192010E9474
S1130BE09508B90180E00E945907B80180E090E0BF
S1130BF00E94AD06180190C091E0F9128DC0809159
S1130C006D0290916E02892B09F488C089EC91E001
S1130C100E946B0B83C062E370E082E00E9459077C
S1130C208091690290916A02209167023091680272
S1130C308217930711F120916D0230916E02232BDC
S1130C4061F09F938F9389ED91E09F938F930E941E
S1130C50550B0F900F900F900F9080916902909117
S1130C606A02892B51F48FEF8F0D823030F481E0CA
S1130C7090E00E944C02E12C01C0EF2C80916902AB
S1130C8090916A02909368028093670280E00E94C8
S1130C90E10082E00E94E100FE14E1F180916D0226
S1130CA090916E02892B01F1EE2DF0E0EE0FFF1F03
S1130CB0E55EFD4F81818F9380818F93EF2DF0E06E
S1130CC0EE0FFF1FE55EFD4F81818F9380818F932F
S1130CD08CEE91E09F938F930E94550B0F900F9091
S1130CE00F900F900F900F90E2E0EE120BC08FEF79
S1130CF09FE00E949A0280E090E00E944C0261E032
S1130D0070E004C0E11006C060E070E082E090E0B2
S1130D100E94AD06FE2CE3CCEF2CFCCF82E0E82E43
S1130D20BDCF9F70FB019083818382E090E00895A2
S1130D30FB0120E4208324E0880F991F2A95E1F722
S1130D409183828383E090E008958CEF8AB996E0E2
S1130D5094B98BB984E085B90895FC01EE0FFF1FA7
S1130D608E0F9F1FFC01EC5CFD4F808121E030E081
S1130D70018002C0220F331F0A94E2F7428150E03F
S1130D80E82FF0E080A14617570711F0282B02C086
S1130D902095282320A308951F920F920FB60F9237
S1130DA01124DF92EF92FF920F931F932F933F939F
S1130DB04F935F936F937F938F939F93AF93BF935F
S1130DC0EF93FF93CF93DF9300D000D0CDB7DEB77E
S1130DD08091B3029091B402909385008093840033
S1130DE0E12CF12C93E0D92E8701000F111F000F85
S1130DF0111F0D581D4FF80180819181892BF1F04D
S1130E0082819381892B31F082819381019793832D
S1130E10828314C019821A821B821C82D982EA82BC
S1130E20BE016F5F7F4F80917102909172020E94A8
S1130E306301892B19F0F80111821082FFEFEF1A78
S1130E40FF0A80E1E816F10479F60F900F900F90F5
S1130E500F90DF91CF91FF91EF91BF91AF919F914F
S1130E608F917F916F915F914F913F912F911F913E
S1130E700F91FF90EF90DF900F900FBE0F901F9097
S1130E80189590937202809371027093B4026093E8
S1130E90B302709385006093840010928000E1E8AF
S1130EA0F0E080818770482B408381E080936F005D
S1130EB008950F931F93CF93C82F8B010E94FC00BA
S1130EC084E0C89FF0011124ED58FD4F1383028381
S1130ED081E090E091838083CF911F910F910C94D6
S1130EE007011F920F920FB60F9211240F900FBE9D
S1130EF00F901F9018951F920F920FB60F92112406
S1130F000F900FBE0F901F9018951F920F920FB65F
S1130F100F9211242F933F934F935F936F937F937B
S1130F208F939F93AF93BF93EF93FF93CF93DF93ED
S1130F3000D000D0CDB7DEB78091C00087FF12C0CB
S1130F408091C60019821A821B821C8291E09983C7
S1130F508A83BE016F5F7F4F8091B5029091B60284
S1130F600E9463010F900F900F900F90DF91CF912B
S1130F70FF91EF91BF91AF919F918F917F916F916D
S1130F805F914F913F912F910F900FBE0F901F9043
S1130F9018954F925F926F927F928F929F92AF9229
S1130FA0BF92CF92DF92EF92FF92CF93DF9300D064
S1130FB000D0CDB7DEB76A017B019093B60280936F
S1130FC0B5024A015B0183E0880C991CAA1CBB1C76
S1130FD08A95D1F760E070E88CEF9AE0A50194015E
S1130FE00E949508CA01B9016B5F7F4F8F4F9F4FD5
S1130FF02AE0422E512C612C712CA30192010E94F3
S1131000950829833A834B835C8334E0CC0CDD1C44
S1131010EE1CFF1C3A95D1F760E070E88CEF9AE083
S1131020A70196010E949508CA01B9016B5F7F4F21
S11310308F4F9F4FA30192010E94950829013A0105
S1131040A501940169817A818B819C810E94850824
S1131050705477FF03C07195619571094B01770F47
S1131060AA08BB08A7019601C301B2010E94850822
S1131070705477FF03C0719561957109CB01770FA7
S1131080AA0BBB0B88169906AA06BB0610F09201A0
S113109007C029813A818091C00082608093C0009A
S11310A0215031092093C4003093C50088E1809316
S11310B0C1008091C10080688093C1000F900F909F
S11310C00F900F90DF91CF91FF90EF90DF90CF9032
S11310D0BF90AF909F908F907F906F905F904F9054
S11310E008959091C00095FFFCCF8093C6000895A9
S11310F0CF93C82F0E947108CA3019F48DE00E9462
S1131100710880E090E0CF910895DB018F939F9365
S11311100E94C608BF91AF91A29F800D911DA39F0D
S1131120900DB29F900D11240895A1E21A2EAA1BCE
S1131130BB1BFD010DC0AA1FBB1FEE1FFF1FA21783
S1131140B307E407F50720F0A21BB30BE40BF50B80
S1131150661F771F881F991F1A9469F76095709509
S1131160809590959B01AC01BD01CF010895A29F8C
S1131170B001B39FC001A39F700D811D1124911D67
S1131180B29F700D811D1124911D08950E94B7080E
S1131190A59F900DB49F900DA49F800D911D1124C7
S11311A008950F931F93CF93DF938230910510F42A
S11311B082E090E0E091C702F091C80220E030E0C4
S11311C0A0E0B0E0309719F1408151810281138190
S11311D048175907C8F08417950769F4109731F038
S11311E012960C93129713961C9327C00093C70270
S11311F01093C80222C02115310519F04217530774
S113120018F49A01BD01EF01DF01F801DBCF2115CC
S11312103105F9F0281B390B2430310580F48A811B
S11312209B816115710521F0FB019383828304C0C6
S11312309093C8028093C702FE01329644C0FE0117
S1131240E20FF31F8193919322503109398328834C
S11312503AC02091C5023091C602232B41F420915B
S11312600201309103013093C6022093C5022091FC
S11312700001309101012115310541F42DB73EB72C
S11312804091040150910501241B350BE091C502E6
S1131290F091C602E217F307A0F42E1B3F0B2817A8
S11312A0390778F0AC014E5F5F4F2417350748F0DB
S11312B04E0F5F1F5093C6024093C50281939193D2
S11312C002C0E0E0F0E0CF01DF91CF911F910F91D8
S11312D00895CF93DF93009709F481C0FC013297FE
S11312E013821282A091C702B091C802109781F4B0
S11312F020813181820F931F2091C5023091C60253
S11313002817390751F5F093C602E093C50267C068
S1131310ED0120E030E0CE17DF0740F44A815B8125
S11313209E0141155105F1F0EA01F5CFD383C28343
S113133040815181840F951FC817D90759F48881BA
S11313409981840F951F0296918380838A819B8162
S1131350938382832115310529F4F093C802E09325
S1131360C7023DC0E901FB83EA8349915991C40F47
S1131370D51FEC17FD0761F480819181840F951FBF
S11313800296E90199838883828193819B838A836E
S1131390E0E0F0E012968D919C911397009719F07C
S11313A0FD01DC01F7CF8D919C9111979D012E5F7A
S11313B03F4F820F931F2091C5023091C602281718
S11313C0390769F4309729F41092C8021092C702C1
S11313D002C013821282B093C602A093C502DF91A9
S11313E0CF910895A0E0B0E0E8EFF9E00C94F40D9B
S11313F05C016B017A016115710519F0FB019183A0
S11314008083E114F10429F0C7010297839708F05F
S1131410E5C0E5012196F5011081812F90E00E943D
S1131420080B892B11F05E01F4CF1D3229F42196AB
S1131430F501118101E007C01B3221F4E501229678
S1131440F501118100E0E114F10409F1F0E1EF1676
S1131450F10429F43FC010E3E114F10421F128E080
S1131460E216F10401F154F4E2E0EE16F10421F580
S1131470812C912CA12CB0E4BB2E3EC0FAE0EF16D7
S1131480F10439F020E1E216F104B1F430C0103374
S113149019F1FAE0EF2EF12CACEC8A2E982CA82C42
S11314A0ACE0BA2E29C078E0E72EF12C812C912CE7
S11314B0A12CE0E1BE2E20C060E070E080E090E866
S11314C097010F2C000C440B550B0E949508490101
S11314D05A0112C0103359F488818F7D883509F080
S11314E0BACF19812296026080E1E82EF12C812C7A
S11314F0912CA12C68E0B62E40E060E070E0CB01B6
S113150027010F2C000C66087708FE0150ED352EDC
S1131510310E29E0231570F42FEB210F2A3118F432
S113152039EC332E06C02FE9210F2A3118F529EAA8
S1131530322E310E232D30E02E153F05DCF447FD0D
S113154016C086169706A806B90670F0A301920184
S11315500E948508630D711D811D911D6130710507
S1131560810520E8920710F04FEF01C041E0219679
S11315701081CBCF202F2170C114D10471F04423EA
S113158029F02197F601D183C08307C001FF19C058
S11315902297F601D183C08314C047FF12C02223CF
S11315A029F060E070E080E090E804C06FEF7FEF26
S11315B08FEF9FE722E230E03093D0022093CF02F6
S11315C009C0222381F090958095709561957F4F95
S11315D08F4F9F4F462F372F282F12C040E030E007
S11315E020E090E00DC097FFF5CF82E290E0909369
S11315F0D0028093CF026FEF7FEF8FEF9FE7EACFA8
S1131600642F732F822FCDB7DEB7E1E10C94100E57
S113161091110C947C0D803219F089508550C8F7D3
S113162008959111089581568A5108F4805285587D
S113163008950F931F93CF93DF93FB01238121FD23
S113164003C08FEF9FEF2CC022FF16C04681578145
S1131650248135814217530744F4A081B1819D014F
S11316602F5F3F4F318320838C93268137812F5FF7
S11316703F4F3783268314C08B01EC01FB010084A8
S1131680F185E02D0995892BE1F6D80116968D9107
S11316909C911797019617969C938E931697CE015B
S11316A0DF91CF911F910F910895A0E0B0E0EBE599
S11316B0FBE00C94030EAE014B5F5F4FFA016191A6
S11316C07191AF018091CB029091CC020E949B0B4F
S11316D0E2E00C941F0E0F931F93CF93DF93E091DE
S11316E0CB02F091CC02238121FF1BC08C01D0E0FE
S11316F0C0E0F80181918F016091CB027091CC021E
S1131700DB011896ED91FC911997882331F0099526
S1131710892B79F3DFEFCFEFECCF8AE00995892BA2
S113172019F08FEF9FEF02C08D2F9C2FDF91CF9187
S11317301F910F910895ABE0B0E0E1EAFBE00C9457
S1131740F30D6C017B018A01FC01178216828381EF
S113175081FFCCC1CE0101963C01F6019381F701D2
S113176093FD859193FF81917F01882309F4BAC188
S1131770853239F493FD859193FF81917F01853200
S113178029F4B60190E00E94190BE7CF912C212C8B
S1131790312CFFE1F315D8F08B3279F038F4803234
S11317A079F08332A1F4232D20611DC08D3261F0C4
S11317B0803369F4232D216016C0832D8260382E76
S11317C0E32DE4603E2E2AC0F32DF8601DC037FCE3
S11317D02DC020ED280F2A3040F08E32B9F436FCAB
S11317E081C1232D2064322E19C036FE06C08AE042
S11317F0989E200D1124922E11C0EAE02E9E200DF9
S11318001124222EF32DF0623F2E08C08C3621F4D1
S1131810832D8068382E02C0883641F4F70193FD89
S1131820859193FF81917F018111B3CF982F9F7D83
S11318309554933028F40C5F1F4F9FE399830DC098
S1131840833631F0833771F0833509F059C021C0F4
S1131850F801808189830E5F1F4F88248394912C23
S1131860530113C02801F2E04F0E511CF801A0806F
S1131870B18036FE03C0692D70E002C06FEF7FEFC8
S1131880C5010E948A0D4C018201F32DFF773F2E82
S113189016C0280122E0420E511CF801A080B1803C
S11318A036FE03C0692D70E002C06FEF7FEFC50103
S11318B00E947F0D4C01F32DF0683F2E820133FC12
S11318C01BC0822D90E088169906B0F4B60180E220
S11318D090E00E94190B2A94F4CFF50137FC85910E
S11318E037FE81915F01B60190E00E94190B21102F
S11318F02A9421E0821A91088114910471F7E8C0B6
S1131900843611F0893641F5F80137FE07C060814D
S11319107181828193810C5F1F4F08C06081718146
S1131920072E000C880B990B0E5F1F4FF32DFF76CB
S11319303F2E97FF09C090958095709561957F4FD4
S11319408F4F9F4FF0683F2E2AE030E0A3010E94A2
S1131950950D882E861845C0853731F4232D2F7EAA
S1131960B22E2AE030E025C0932D997FB92E8F3610
S1131970C1F018F4883579F0B5C0803719F088378C
S113198021F0B0C0E92FE061BE2EB4FE0DC0FB2DE6
S1131990F460BF2E09C034FE0AC0292F2660B22E7F
S11319A006C028E030E005C020E130E002C020E1BC
S11319B032E0F801B7FE07C06081718182819381B2
S11319C00C5F1F4F06C06081718180E090E00E5F64
S11319D01F4FA3010E94950D882E8618FB2DFF77BB
S11319E03F2E36FE0DC0232D2E7FA22E891458F4CF
S11319F034FE0BC032FC09C0832D8E7EA82E05C098
S1131A00B82CA32C03C0B82C01C0B92CA4FE0FC061
S1131A10FE01E80DF11D8081803321F49A2D997E19
S1131A20A92E09C0A2FE06C0B394B39404C08A2DA3
S1131A30867809F0B394A3FC11C0A0FE06C0B214CA
S1131A4088F4280C922C9B180EC0B21460F4B601D2
S1131A5080E290E00E94190BB394F7CFB21418F40B
S1131A602B1802C0982C212CA4FE10C0B60180E3D0
S1131A7090E00E94190BA2FE17C0A1FC03C088E7E6
S1131A8090E002C088E590E0B6010CC08A2D86780B
S1131A9059F0A1FE02C08BE201C080E2A7FC8DE2F6
S1131AA0B60190E00E94190B891438F4B60180E362
S1131AB090E00E94190B9A94F7CF8A94F301E80DF1
S1131AC0F11D8081B60190E00E94190B8110F5CFC1
S1131AD0222009F442CEB60180E290E00E94190B64
S1131AE02A94F6CFF6018681978102C08FEF9FEF8B
S1131AF02B96E2E10C940F0E992788270895FC0198
S1131B000590615070400110D8F7809590958E0F24
S1131B109F1F0895FC016150704001900110D8F797
S1131B20809590958E0F9F1F0895FA01AA2728305B
S1131B3051F1203181F1E8946F936E7F6E5F7F4F96
S1131B408F4F9F4FAF4FB1E03ED0B4E03CD0670F12
S1131B50781F891F9A1FA11D680F791F8A1F911D65
S1131B60A11D6A0F711D811D911DA11D20D009F4B5
S1131B7068943F912AE0269F11243019305D3193F7
S1131B80DEF6CF010895462F4770405D4193B3E0E0
S1131B900FD0C9F7F6CF462F4F70405D4A3318F087
S1131BA0495D31FD4052419302D0A9F7EACFB4E038
S1131BB0A6959795879577956795BA95C9F70097F0
S1131BC06105710508959B01AC010A2E0694579591
S1131BD0479537952795BA95C9F7620F731F841FE8
S1131BE0951FA01D08952F923F924F925F926F927E
S1131BF07F928F929F92AF92BF92CF92DF92EF9299
S1131C00FF920F931F93CF93DF93CDB7DEB7CA1B19
S1131C10DB0B0FB6F894DEBF0FBECDBF09942A8844
S1131C20398848885F846E847D848C849B84AA84EC
S1131C30B984C884DF80EE80FD800C811B81AA8179
S1131C40B981CE0FD11D0FB6F894DEBF0FBECDBF44
S10B1C50ED010895F894FFCFA3
S1131C580000D10220000000000200000000780803
S1131C680000000068016C01436F6E764669666F78
S1131C78004572726F72204932435F535441525483
S1131C88004572726F72204932435F534C415F4181
S1131C98434B004572726F72204932435F4441548A
S1131CA8415F41434B0053657420737769746368DB
S1131CB820746F2025730A004F4646004F4E005388
S1131CC8657420506F77657220746F2025752064C1
S1131CD869676974730A0025732025730A004F4BDA
S1131CE83A2530347500494E56414C4944205354E2
S1131CF8415445004F4B3A2575004F4B3A25640033
S1131D084F4B004F4B3A257300554E4B4E4F574E91
S1131D1820434F4D4D414E440052656D6F7465200C
S1131D2874696D656F75742100507772537769749F
S1131D3863685F696E203D2025640A0053746174EA
S1131D4865206368616E67652022257322203D3E05
S1131D5820222573220A004E6F726D616C00526551
S1131D686D6F7465004572726F720007020E02157A
S1131D780276312E310048656E64692D436F6E74A6
S1131D88726F6C000502010B06010B07010B0201BF
S10F1D980B03010B04010B050105010104
S9030000FC
